:100000000C9489030C94A6030C94A6030C94592613
:100010000C9449120C94A6030C94A6030C9484151A
:100020000C94A6030C94A6030C94A6030C94A603AC
:100030000C94A6030C94A6030C94A6030C94A6039C
:100040000C94E1140C94A6030C94F7110C94B011C9
:100050000C94A6030C94A6030C94A6030C94A6037C
:100060000C94A6030C94A6034D194D194D1964194F
:10007000791982198B1994199D19B419C019C919C4
:10008000D219DB19ED19011A131A291A3B1A441A4D
:100090004D1A561A611A084AD73B3BCE016E84BCF2
:1000A000BFFDC12F3D6C74319ABD56833DDA3D00D2
:1000B000C77F11BED9E4BB4C3E916BAAAABE00001B
:1000C00000803F05A84CCDB2D44EB93836A9020CF9
:1000D00050B9918688083CA6AAAA2ABE00000080D2
:1000E0003F3E0D0A002C0057506F733A002C002C35
:1000F0004D506F733A003C436865636B003C416C44
:1001000061726D003C486F6D65003C486F6C640027
:100110003C52756E003C5175657565003C49646CD8
:1001200065000D0A003D00244E005D0D0A002046CA
:1001300000205400204D3800204D3900204D35005E
:10014000204D3400204D3300204D3200204D310031
:10015000204D3000204739340020473933002047F4
:1001600039310020473930002047323100204732F2
:1001700030002047313900204731380020473137DF
:10018000002047005B473830005B4733005B473255
:10019000005B4731005B4730005D0D0A002C005BBF
:1001A0004739323A005D0D0A002C0033303A0032F4
:1001B000383A0035393A0035383A0035373A0035A3
:1001C000363A0035353A0035343A005B470020288E
:1001D000686F6D696E672070756C6C2D6F66662C2C
:1001E000206D6D290D0A002028686F6D696E6720EB
:1001F0006465626F756E63652C206D736563290D90
:100200000A2432323D002028686F6D696E672073C2
:1002100065656B2C206D6D2F6D696E290D0A24327A
:10022000313D002028686F6D696E672066656564E2
:100230002C206D6D2F6D696E290D0A2432303D0022
:10024000290D0A2431393D002028686F6D696E67D9
:100250002064697220696E76657274206D61736BBB
:100260002C20696E743A002028686F6D696E6720D3
:100270006379636C652C20626F6F6C290D0A2431E1
:10028000383D00202868617264206C696D69747360
:100290002C20626F6F6C290D0A2431373D00202815
:1002A000696E76657274207374657020656E616224
:1002B0006C652C20626F6F6C290D0A2431363D006D
:1002C00020286175746F2073746172742C20626FC2
:1002D0006F6C290D0A2431353D0020287265706F3E
:1002E000727420696E636865732C20626F6F6C296D
:1002F0000D0A2431343D0020286E2D646563696D3C
:10030000616C732C20696E74290D0A2431333D0011
:1003100020286E2D61726320636F72726563746949
:100320006F6E2C20696E74290D0A2431323D002035
:10033000286172632C206D6D2F7365676D656E7417
:10034000290D0A2431313D0020286A756E637469D5
:100350006F6E20646576696174696F6E2C206D6DB7
:10036000290D0A2431303D002028616363656C65E6
:10037000726174696F6E2C206D6D2F7365635E32D0
:10038000290D0A24393D00202873746570206964A2
:100390006C652064656C61792C206D736563290D33
:1003A0000A24383D00290D0A24373D0020287374A3
:1003B000657020706F727420696E76657274206D3E
:1003C00061736B2C20696E743A0020286465666145
:1003D000756C74207365656B2C206D6D2F6D696E67
:1003E000290D0A24363D00202864656661756C7409
:1003F00020666565642C206D6D2F6D696E290D0A70
:1004000024353D002028737465702070756C736509
:100410002C2075736563290D0A24343D0020287A49
:100420002C20737465702F6D6D290D0A24333D00E7
:100430002028792C20737465702F6D6D290D0A2486
:10044000323D002028782C20737465702F6D6D2943
:100450000D0A24313D0024303D00242420287669F3
:100460006577204772626C2073657474696E677378
:10047000290D0A24232028766965772023207061BE
:1004800072616D6574657273290D0A2447202876A0
:100490006965772070617273657220737461746529
:1004A000290D0A244E2028766965772073746172BD
:1004B00074757020626C6F636B73290D0A24783D2C
:1004C00076616C7565202873617665204772626C71
:1004D0002073657474696E67290D0A244E783D6C2B
:1004E000696E652028736176652073746172747516
:1004F0007020626C6F636B290D0A244320286368A7
:1005000065636B2067636F6465206D6F6465290D9B
:100510000A245820286B696C6C20616C61726D2014
:100520006C6F636B290D0A2448202872756E206851
:100530006F6D696E67206379636C65290D0A7E2093
:10054000286379636C65207374617274290D0A21C4
:1005500020286665656420686F6C64290D0A3F2059
:100560002863757272656E74207374617475732973
:100570000D0A6374726C2D7820287265736574207F
:100580004772626C290D0A000D0A4772626C2030B6
:100590002E3961205B27242720666F722068656CE6
:1005A000705D0D0A005D0D0A0044697361626C653F
:1005B0006400456E61626C65640043617574696FC7
:1005C0006E3A20556E6C6F636B6564002724482774
:1005D0007C2724582720746F20756E6C6F636B0026
:1005E000526573657420746F20636F6E74696E75E5
:1005F00065005B002E204D506F733F0D0A00416275
:100600006F727420647572696E67206379636C65BC
:100610000048617264206C696D697400414C4152FC
:100620004D3A20000D0A00416C61726D206C6F63C1
:100630006B0042757379206F722071756575656402
:1006400000454550524F4D207265616420666169D6
:100650006C2E205573696E672064656661756C74D5
:10066000730056616C7565203C203320757365639B
:100670000056616C7565203C20302E300053657447
:1006800074696E672064697361626C656400496EA9
:1006900076616C69642073746174656D656E740055
:1006A0004D6F64616C2067726F75702076696F6C36
:1006B0006174696F6E00496E76616C696420726165
:1006C0006469757300556E737570706F72746564CC
:1006D0002073746174656D656E7400457870656330
:1006E00074656420636F6D6D616E64206C657474F5
:1006F000657200426164206E756D62657220666F7E
:10070000726D6174006572726F723A20006F6B0DCA
:100710000A0011241FBECFEFD8E0DEBFCDBF11E02D
:10072000A0E0B1E0EAEEF2E602C005900D92A03042
:10073000B107D9F716E0A0E0B1E001C01D92A739DA
:10074000B107E1F70E94A8030C9473310C940000E8
:100750000F931F930E947D110E94691B0E945C15DC
:10076000789480E1ECE5F5E0DF011D928A95E9F7E8
:1007700081E080935C0580935D0506E011E0809147
:100780005C05882389F10E94F2110E9469220E946F
:1007900013110E949F140E9441110E9465110E9432
:1007A000BF230E9433150E94C72210925C0510924D
:1007B0005E0580918406982F81FF02C010936B051F
:1007C00080915D05813021F494FF02C000935D05A6
:1007D00080915D05863021F482E00E94002804C0EB
:1007E00010925D050E94E6120E9485120E9450142C
:1007F000C6CF80915E0584FD15C080915E05806145
:1008000080935E050E9447110E946A1180915D05E8
:100810008350833038F480915E05806280935E055A
:100820000E9441150895EF92FF920F931F93CF936B
:10083000DF937B018C0120E030E040EA51E40E942C
:1008400058300E94552E0E94EC2DEB010E944C2244
:10085000C801B70120E030E04AE754E40E94583074
:100860007B018C0182E390E0C89FB001C99F700DAD
:10087000D89F700D112480E090E00E94182E9B01FB
:10088000AC01C801B7010E949E2C0E94552E0E9407
:10089000EC2DDC01CB010E947D2200E911E00EC0AD
:1008A0000E94851280915C05882351F484EF91E0C9
:1008B000F8013197F1F70197D9F72197209781F740
:1008C000DF91CF911F910F91FF90EF9008954F927C
:1008D0005F926F927F928F92AF92BF92CF92DF9290
:1008E000EF92FF920F931F93DF93CF9300D000D02E
:1008F000CDB7DEB72B013C0129833A834B835C8360
:1009000080915D058730F9F00E94851280915C0529
:100910008823C9F40E94EF1B8823B1F7C301B201F9
:1009200029813A814B815C810E94841E80915D0502
:10093000882319F482E080935D0580916B058823FC
:1009400011F00E94F7140F900F900F900F90CF911D
:10095000DF911F910F91FF90EF90DF90CF90BF90AC
:10096000AF908F907F906F905F904F9008952F92EF
:100970003F924F925F926F927F928F929F92AF922F
:10098000BF92CF92DF92EF92FF920F931F9385E079
:1009900080935D0580916B00817F80936B000E9446
:1009A000FF2580915C05882309F070C08CE0EFE59D
:1009B000F5E0DF011D928A95E9F70E94C7221092A7
:1009C0005D0530918506232F35FD02C06FEF01C014
:1009D00061E026FD03C0DD24DA9402C0DD24D39457
:1009E00037FD03C0CC24CA9402C0CC24C394E09049
:1009F0009006F09091060091920610919306772749
:100A000067FD7095872F972F0E941A2EA8019701D6
:100A10000E9458301B012C016D2D772767FD7095C2
:100A2000872F972F0E941A2EA80197010E945830F5
:100A30003B014C016C2D772767FD7095872F972F11
:100A40000E941A2EA80197010E9458307B018C0148
:100A5000A0908A06B0908B06C0908C06D0908D0630
:100A6000C201B101A401930188240E9467040E947D
:100A7000F7140E944C220E94C7228091840683FFB3
:100A800005C080916B008E6080936B001F910F9169
:100A9000FF90EF90DF90CF90BF90AF909F908F909E
:100AA0007F906F905F904F903F902F9008952F927E
:100AB0003F924F925F926F927F928F929F92AF92EE
:100AC000BF92CF92DF92EF92FF920F931F93DF932B
:100AD000CF93CDB7DEB7CE54D0400FB6F894DEBF7B
:100AE0000FBECDBF3C017EAF6DAF21965FAF4EAF65
:100AF000219722962FAF229723960FAF2397249604
:100B0000EFAE24972896ACAEBDAECEAEDFAE289742
:100B100029968FAE2997E22EFF24EE0CFF1CEE0CD7
:100B2000FF1C4E0D5F1D5CAF4BAFDA012D903D9069
:100B30004D905C90FC01EE0DFF1DC201B1012081C2
:100B40003181428153810E949F2C69AB7AAB8BAB80
:100B50009CAB10E0000F111F000F111F2196EEAD8E
:100B6000FFAD2197E00FF11FFAAFE9AFA080B18090
:100B7000C280D380F301E00FF11FC601B5012081CF
:100B80003181428153810E949F2C6DA77EA78FA740
:100B900098AB24962FAD2497E22FF0E0EE0FFF1FC5
:100BA000EE0FFF1F6E0E7F1ED3018D919D910D9054
:100BB000BC91A02D8DAB9EABAFABB8AF2DAD3EAD14
:100BC000E20FF31F60817181828193812DA93EA97B
:100BD0004FA958AD0E949E2C69A77AA78BA79CA706
:100BE000D201C101B0588DA39EA3AFA3B8A7A6019F
:100BF0009501505829A33AA34BA35CA34DAD5EAD1C
:100C0000E40EF51ED7016D917D918D919C9129A9DE
:100C10003AA94BA95CA90E949E2C3B014C01EDAD69
:100C2000FEAD0E0F1F1FD8016D917D918D919C918E
:100C30002DA53EA54FA558A90E949E2C5B016C01D5
:100C40006DA17EA18FA198A5A60195010E945830A3
:100C50007B018C0169A17AA18BA19CA1A4019301C4
:100C60000E9458309B01AC01C801B7010E949E2C24
:100C70001B012C016DA17EA18FA198A5A401930158
:100C80000E9458307B018C0169A17AA18BA19CA1A3
:100C9000A60195010E9458309B01AC01C801B70123
:100CA0000E949F2C9B01AC01C201B1010E94122D38
:100CB0005B016C01A8968FADA897882399F0C601B7
:100CC000B50120E030E040E050E00E94862F88230C
:100CD000ECF0C601B5012BED3FE049EC50E40E9479
:100CE0009E2C12C0C601B50120E030E040E050E08B
:100CF0000E94782D181654F0C601B5012BED3FE087
:100D000049EC50E40E949F2C5B016C01C601B501C7
:100D1000A7962CAD3DAD4EAD5FADA7970E94583064
:100D200029A53AA54BA55CA50E94932F7B018C01B8
:100D300020E030E040E050E00E94782D882309F464
:100D4000D5C1C801B701209178063091790640914C
:100D50007A0650917B060E947F2D0E94552E0E949C
:100D6000EC2D78A36F8F2996BFAD2997BB23A1F0F7
:100D700080E090E00E94182E9B01AC0128966CAD9B
:100D80007DAD8EAD9FAD28970E94583028966CAFF0
:100D90007DAF8EAF9FAF28972F8D38A1B90180E02E
:100DA00090E00E94182E7B018C01C601B501A801BC
:100DB00097010E947F2D6B8F7C8F8D8F9E8F69A5F1
:100DC0007AA58BA59CA5A80197010E947F2D6F8B0A
:100DD000788F898F9A8F6B8D7C8D8D8D9E8D20E085
:100DE00030E040E05FEB0E9458302B8D3C8D4D8D04
:100DF0005E8D0E94583020E030E040E85FE30E94C2
:100E00009F2C6B8B7C8B8D8B9E8B24963FAD249778
:100E1000E32FF0E0EE0FFF1FEE0FFF1FCE01019654
:100E2000E80FF91F2DA93EA94FA958AD20833183A2
:100E30004283538341E050E05E874D8766242296CB
:100E4000BFAD2297AB2FB0E0AA0FBB1FAA0FBB1FED
:100E5000A80FB91F2B96BFAFAEAF2B9723963FAD10
:100E60002397232F30E0220F331F220F331F280F29
:100E7000391F2D963FAF2EAF2D972F96FFAFEEAFB8
:100E80002F970EC1262D332727FD3095809196068A
:100E900090E0281739070CF046C06DA17EA18FA104
:100EA00098A52B8D3C8D4D8D5E8D0E9458307B0119
:100EB0008C0169A17AA18BA19CA12B893C894D89C8
:100EC0005E890E9458309B01AC01C801B7010E94A5
:100ED0009F2C7B018C016DA17EA18FA198A52B89F0
:100EE0003C894D895E890E9458305B016C0169A183
:100EF0007AA18BA19CA12B8D3C8D4D8D5E8D0E9486
:100F000058309B01AC01C601B5010E949E2C6DA317
:100F10007EA38FA398A76394C701D80189A39AA33E
:100F2000ABA3BCA361C04D855E85BA0180E090E0B3
:100F30000E94182E2B8D3C8D4D8D5E8D0E94583059
:100F40007B018C01C8010E947C2D6F87788B898B77
:100F50009A8BB701C8010E94DB303B014C01ABAD5D
:100F6000BCADED90FD900D911C9117FB109517F9FC
:100F70001095E9ADFAAD2080318042805380C801E0
:100F8000B7012F85388949895A890E9458305B01F9
:100F90006C01C201B101A40193010E9458309B0170
:100FA000AC01C601B5010E949F2C6DA37EA38FA347
:100FB00098A7C801B701A40193010E9458307B0192
:100FC0008C01C201B1012F85388949895A890E9453
:100FD00058309B01AC01C801B7010E949E2C69A347
:100FE0007AA38BA39CA3662469A97AA98BA99CA93F
:100FF0002DA13EA14FA158A50E949F2C2B96AEADCE
:10100000BFAD2B976D937D938D939C9313976DA597
:101010007EA58FA598A929A13AA14BA15CA10E9408
:101020009F2C2D96EEADFFAD2D976083718382834B
:1010300093832F96AEADBFAD2F976D917D918D911E
:101040009C912F89388D498D5A8D0E949F2C2F9607
:10105000EEADFFAD2F9760837183828393836981A7
:101060007A818B819C812D813E814F815885E984D5
:10107000FA840B851C852896ACACBDACCEACDFAC3D
:10108000289729968FAC29970E94670480915C0568
:10109000882361F52D853E852F5F3F4F3E872D8745
:1010A0004D855E858F8D98A14817590708F4EACEC3
:1010B000ADADBEAD6D917D918D919C9113971496C0
:1010C0002D913D914D915C9117971896ED90FD9063
:1010D0000D911C911B972896ACACBDACCEACDFAC8F
:1010E000289729968FAC29970E946704C25BDF4F2F
:1010F0000FB6F894DEBF0FBECDBFCF91DF911F9129
:101100000F91FF90EF90DF90CF90BF90AF909F90A6
:101110008F907F906F905F904F903F902F900895A9
:10112000AF92BF92CF92DF92EF92FF920F931F93F5
:1011300059016A010E941A2E2091610630916206BF
:1011400040916306509164060E947F2D609378055C
:101150007093790580937A0590937B05C601B5015C
:101160000E941A2E2091650630916606409167060E
:10117000509168060E947F2D60937C0570937D05D9
:1011800080937E0590937F05C801B7010E941A2EB7
:101190002091690630916A0640916B0650916C0669
:1011A0000E947F2D60938005709381058093820556
:1011B000909383051F910F91FF90EF90DF90CF9058
:1011C000BF90AF9008952F923F924F925F926F928F
:1011D0007F928F929F92AF92BF92CF92DF92EF92C7
:1011E000FF920F931F93DF93CF93CDB7DEB7EE97A8
:1011F0000FB6F894DEBF0FBECDBF3C0180915D05F8
:10120000863011F48CE0B9C719828CE0FE01369665
:10121000DF01482F1D924A95E9F7FE017296DF0122
:101220001D928A95E9F710926C05442455242224D6
:101230001AAE33243A94A3E0AA2EF2E0BF2E01E0C6
:10124000E1E08E2E912CA5C12E313105C9F12F314F
:101250003105D4F42431310584F421313105A4F56C
:101260002430310569F1253031051CF437FF2AC0DF
:1012700025C02A30310511F523C02631310554F13E
:101280002C313105D9F41CC02C3531058CF42A35AC
:101290003105E4F42C3331053CF426333105E4F414
:1012A0002533310559F40CC02035310539F40AC015
:1012B0002C35310529F02F35310554F010E00DC0E3
:1012C00011E00BC012E009C013E007C014E005C034
:1012D00016E003C017E001C019E02531310509F41B
:1012E00094C026313105A4F52430310509F467C0D6
:1012F00025303105A4F42130310509F465C02230D0
:10130000310524F4232B09F45CC02EC122303105B1
:1013100009F45DC02330310509F026C15BC02231DC
:10132000310509F461C0233131054CF42A3031050F
:1013300009F443C02131310509F016C14EC02331F3
:10134000310509F458C02431310509F00DC15AC0E6
:101350002035310509F491C021353105ACF4253330
:10136000310509F482C0263331054CF42C313105A6
:1013700009F44EC02E31310509F0F6C049C02C33B6
:1013800031050CF0F1C074C02C35310509F47FC073
:101390002D3531054CF42A35310509F472C02B3551
:1013A000310509F0E1C070C02D35310509F489C05F
:1013B0002E35310509F0D8C087C0B2E04EC0E1E05B
:1013C0004FC010926D05D2C000936D05CFC0B09292
:1013D0006D05CCC0A0926D05C9C010928505009323
:1013E0008605B0928705C2C010928505B092860529
:1013F00000938705BBC000938505B09286051092C7
:101400008705B4C000936F05B1C010926F05AEC0E0
:10141000C701B60120E030E040E251E40E945830BC
:101420000E9432310E94E72DF1E069317F0791F08F
:1014300041E06A3174072CF46851714009F094C09E
:101440000BC081E06C32780751F06D52714009F0A9
:101450008BC008C0A4E033C0B3E0BAAF87C0E5E0FA
:10146000EAAF84C0F6E0FAAF81C0222423947EC0A4
:10147000822F86538093880579C044E040936D05A0
:1014800075C00093700572C0109270056FC0C701DF
:10149000B60120E030E040E251E40E9458300E9462
:1014A00032310E94E72D53E06839750739F06959E8
:1014B000734009F059C098E09AAF58C0A7E0AAAFAE
:1014C00055C000936E0552C010926E054FC0263075
:1014D000310534F42330310554F4772334F403C058
:1014E0002E31310511F010E003C015E001C018E005
:1014F0002430310569F12530310584F4213031057E
:10150000A9F1223031051CF4232BC9F02DC0223063
:101510003105C1F02330310539F517C028303105C8
:10152000E9F02930310524F425303105E9F413C000
:1015300029303105B1F02E313105B1F403C00093EB
:10154000710514C0B092710511C0009372050EC0F0
:10155000309272050BC01092720508C0009373059B
:1015600005C01092730502C0A0926C05112389F08A
:10157000940102C0220F331F1A95E2F7C90184219A
:101580009521892B21F0B5E0B0936C0502C0422A69
:10159000532A9981F301E90FF11D10811123B9F04C
:1015A000812F81548A3110F082E00FC09F5F9983B0
:1015B000C301BE016F5F7F4FAE014E5F5F4F0E9460
:1015C0000423892B09F0F2C581E080936C0580919A
:1015D0006C05882309F0D1C5198299241BAE1CAE75
:1015E000E0E8EDAFFFEBFEAF0F2EF0E0AF2EF0E046
:1015F000BF2EF0E0CF2EF0E0DF2EF02DAEAABFAA76
:10160000C8AED9AE882476E0372E10C1EA80FB80C0
:101610000C811D81C801B70120E030E040E050E0BE
:101620000E94782D181614F030926C0580916E058A
:10163000882381F080916F05882309F4F1C0C801E7
:10164000B70123E333E34BEC51E40E9458307B01B4
:101650008C01E6C080916F05882351F0C801B70165
:1016600023E333E34BEC51E40E9458307B018C01BF
:10167000E0927405F0927505009376051093770556
:10168000C9C02A813B814C815D8180916F0588238F
:1016900051F0CA01B90123E333E34BEC51E40E945A
:1016A00058309B01AC01E12FFF27E7FDF095E9548D
:1016B000F040EE0FFF1FEE0FFF1F61E070E06C0FB8
:1016C0007D1FE60FF71F218B328B438B548BA2C0FB
:1016D0006A817B818C819D810E9432310E94EC2D38
:1016E000862E98C0AA80BB80CC80DD8093C08A8182
:1016F0009B81AC81BD818EAB9FABA8AFB9AF809110
:101700006F05882309F486C06EA97FA988AD99ADBD
:1017100023E333E34BEC51E40E9458306EAB7FABD4
:1017200088AF99AF77C06A817B818C819D8120E0F1
:1017300030E040E050E00E94782D88230CF06AC031
:1017400030926C0567C0EA80FB800C811D81C80166
:10175000B70120E030E040E050E00E94782D88237F
:1017600014F430926C05C801B7010E9432310E9416
:10177000EC2D609384054EC02A813B814C815D81B4
:1017800080916F05882351F0CA01B90123E333E347
:101790004BEC51E40E9458309B01AC012E833F83F7
:1017A0004887598791E0992A35C02A813B814C812D
:1017B0005D8180916F05882351F0CA01B90123E34F
:1017C00033E34BEC51E40E9458309B01AC012A8773
:1017D0003B874C875D87A2E09A2A1CC02A813B8107
:1017E0004C815D8180916F05882351F0CA01B90158
:1017F00023E333E34BEC51E40E9458309B01AC01EE
:101800002E873F87488B598BB4E09B2A03C0E3E0C7
:10181000E0936C058BAD9CADADADBEAD7C018D0193
:10182000D801C701EBAE9CAFADAFBEAF9981F3015C
:10183000E90FF11D10811123B9F0812F81548A31F4
:1018400010F082E00FC09F5F9983C301BE016F5FFC
:101850007F4FAE014E5F5F4F0E940423892B09F03A
:10186000B7C481E080936C0580916C05882309F0F2
:1018700084C480915D05873041F0809172050E949B
:101880004911809173050E946C1151FE13C08E01A5
:10189000025E1F4F80918805B8010E943E1B88237D
:1018A00009F46AC4A9E8B5E0F8018CE001900D9252
:1018B0008150E1F7FAADF43009F45DC1F53048F438
:1018C000F23051F1F33008F0AAC0F13009F0ABC1A9
:1018D0000EC04AAD463009F44EC1463008F49FC0F0
:1018E000473009F453C1483009F09DC193C1C60186
:1018F000B50120E030E040E050E00E94782D8823E0
:101900000CF446C180915D05873009F48CC1C60195
:10191000B5010E94130487C152E0851619F064E1F5
:10192000861651F4C601B5010E9432310E94E72D9E
:10193000CB010197069720F083E080936C0572C17C
:10194000992021F482E0881609F422C17B010894D1
:10195000E108F10894E18916B1F48E2D68E775E08D
:101960000E94331B8091880590E08E159F0509F039
:1019700059C1E9E8F5E0DF0151978CE00D90019243
:101980008150E1F74FC18E2C3EE1A32EB12CAC0E5D
:10199000BD1E8E2DB5010E943E1B882309F4ECC3A9
:1019A00000E010E040E050E0C92CDD24BE016A5F99
:1019B0007F4FC601002E02C0959587950A94E2F7E5
:1019C00080FF0FC09501240F351FFB01E40FF51FA9
:1019D00080819181A281B381F90180839183A28367
:1019E000B3830F5F1F4F4C5F5F4F0330110509F743
:1019F0008E01025E1F4F882DB8010E94331B80911B
:101A0000880590E08E159F0509F00CC1A9E8B5E0A6
:101A1000F8018CE001900D928150E1F703C199200B
:101A200009F478C08E010A5F1F4F28E7E22E25E0F7
:101A3000F22ECC24DD24A92CBB24C5010C2C02C021
:101A4000959587950A94E2F780FF35C080917005DF
:101A50008823F9F0D70151966D917D918D919C91DC
:101A600054975D962D913D914D915C9190970E9478
:101A70009F2C9B01AC01F80160817181828193816F
:101A80000E949F2CD8016D937D938D939C93139707
:101A90001CC0F8016081718182819381D7012D91F1
:101AA0003D914D915C910E949F2CF8016083718360
:101AB000828393830AC0F70180819181A281B381DF
:101AC000F80180839183A283B3830894C11CD11C45
:101AD0000C5F1F4F44E050E0E40EF51E53E0C516C6
:101AE000D10409F0AACF6E817F81888599852A85E6
:101AF0003B854C855D85EE84FF8408891989A0901B
:101B00007306B0907406C0907506D090760688244F
:101B10000E9467046AAD653011F487E001C086E079
:101B20009AE2692E712C6C0E7D1EB3010E943E1B41
:101B3000882309F421C36AA57BA58CA59DA52EA5A4
:101B40003FA548A959A9EAA8FBA80CA91DA9A090DE
:101B50007306B0907406C0907506D09076068824FF
:101B60000E946704A8E7B5E0F3018CE001900D92B4
:101B70008150E1F757C07AAD763011F487E001C0AB
:101B800086E068E775E00E94331B4DC0992021F480
:101B900086E080936C0547C008E715E086E0C82E14
:101BA000D12CCC0EDD1EEE24FF24A92CBB24C501B4
:101BB0000E2C02C0959587950A94E2F780FF1CC011
:101BC000D8016D917D918D919C91139751962D9196
:101BD0003D914D915C9154970E949E2CF60120817D
:101BE0003181428153810E949E2CD8015D966D9374
:101BF0007D938D939C9390970894E11CF11C0C5F4E
:101C00001F4FE4E0F0E0CE0EDF1EF3E0EF16F1042C
:101C100071F608C08CE0E5E9F5E0DF011D928A95D8
:101C2000E9F701C0992442FC03C0992009F490C24D
:101C300080916E05882399F06BAD7CAD8DAD9EAD26
:101C400020E030E040E050E00E94782D88233CF412
:101C500080916D05843019F086E080936C05222018
:101C600039F080916D05823018F086E080936C0524
:101C700080916C05882309F080C28E010A5F1F4F96
:101C8000B8E7EB2EB5E0FB2ECC24DD24A92CBB2439
:101C9000C5010C2C02C0959587950A94E2F780FF48
:101CA00033C02220D9F5809170058823D1F0F70147
:101CB0006189728983899489258D368D478D50A1DC
:101CC0000E949F2C9B01AC01D8016D917D918D915B
:101CD0009C910E949F2CF80160837183828393837F
:101CE0001DC0D8016D917D918D919C91F70120814E
:101CF0003181428153810E949F2CD8016D937D9345
:101D00008D939C9313970AC0F70180819181A281E2
:101D1000B381F80180839183A283B3830894C11CAB
:101D2000D11C0C5F1F4F44E050E0E40EF51E53E061
:101D3000C516D10409F0ACCF80916D05843048F40C
:101D4000823008F04CC0882359F0813009F0F3C18B
:101D500020C0843009F0EFC1992009F4ECC18BC098
:101D6000992009F488C06E817F81888599852A85AC
:101D70003B854C855D85EE84FF8408891989A09098
:101D80007306B0907406C0907506D09076068824CD
:101D900023C0992009F46FC06E817F818885998561
:101DA0002A853B854C855D85EE84FF8408891989E9
:101DB00080906E05882061F4A0917405ABAFB0915E
:101DC0007505BCAFE0917605EDAFF0917705FEAFFC
:101DD000ABACBCACCDACDEAC0E946704ACC181E066
:101DE00090E00090870502C0880F991F0A94E2F7DF
:101DF0008095982209F43FC06EA97FA988AD99AD5E
:101E000020E030E040E050E00E94782D882309F087
:101E100043C0E0918505F0E0EE0FFF1FEE0FFF1FBE
:101E20008E010F5F1F4FE00FF11FC188D288E3883A
:101E3000F488C701B60120E030E040E050E00E94A5
:101E4000782D8823E1F48091860590E0880F991F12
:101E5000880F991F080F191FD80151966D917D9118
:101E60008D919C91549720E030E040E050E00E943A
:101E7000782D882321F486E080936C055CC16EA9DF
:101E80007FA988AD99AD20E030E040E050E00E94AD
:101E9000782D882309F4F8C0E0918505F0E0EE0F75
:101EA000FF1FEE0FFF1F8E010F5F1F4FD801AE0FF8
:101EB000BF1FE858FA4F15966D917D918D919C91B9
:101EC000189720813181428153810E949E2C1B01F1
:101ED0002C01E0918605F0E0EE0FFF1FEE0FFF1FD3
:101EE0000E0F1F1FE858FA4FD80115966D917D917E
:101EF0008D919C91189720813181428153810E945C
:101F00009E2C3B014C018CE0FE017296DF011D927C
:101F10008A95E9F76EA97FA988AD99AD20E030E0F8
:101F200040E850E40E9458302EA93FA948AD59AD71
:101F30000E9458307B018C01C201B101A2019101C4
:101F40000E9458309B01AC01C801B7010E949E2C31
:101F50007B018C01C401B301A40193010E9458309C
:101F60009B01AC01C801B7010E949E2C7B018C0132
:101F700020E030E040E050E00E94782D882324F4F7
:101F800084E080936C05F9C0C801B7010E94E53078
:101F90007B018C01C201B101A40193010E94932F26
:101FA0009B01AC0117FB109517F91095C801B701FB
:101FB0000E947F2D6B017C0180916D05833021F49F
:101FC000F7FAF094F7F8F0946EA97FA988AD99AD6F
:101FD00020E030E040E050E00E94782D88236CF44F
:101FE000F7FAF094F7F8F0944EA95FA968AD79ADCF
:101FF00070584EAB5FAB68AF79AF00918505A02EEE
:10200000BB24AA0CBB1CAA0CBB1C8E010F5F1F4F6C
:10201000A00EB11EC401B301A70196010E94583061
:102020009B01AC01C201B1010E949E2C20E030E076
:1020300040E05FE30E945830D50151966D937D9347
:102040008D939C9354978091860590E0880F991FFB
:10205000880F991F080F191FC201B101A70196012E
:102060000E9458309B01AC01C401B3010E949F2C17
:1020700020E030E040E05FE30E945830F801618BDF
:10208000728B838B948B15C0E0918605F0E0EE0F88
:10209000FF1FEE0FFF1FEC0FFD1F228933894489BC
:1020A0005589C701B6010E94932F6EAB7FAB88AFF5
:1020B00099AF90916D052091850500918605E0907E
:1020C000870580906E05882061F4F0917405FBAF60
:1020D000409175054CAF509176055DAF60917705E5
:1020E0006EAF00D000D00F92EDB7FEB731964EA97B
:1020F0005FA968AD79ADADB7BEB711964D935D934D
:102100006D937C93149780E0923009F481E084838E
:1021100088E795E0BE016A5F7F4FAE014E5E5F4F7C
:10212000ABACBCACCDACDEAC0E9457050F900F90B1
:102130000F900F900F9080916C058823F1F4A8E721
:10214000B5E0FE0136968CE001900D928150E1F7EA
:1021500080917105882369F00E944C2210926B05D2
:1021600080917105823019F40E94F90302C0109227
:10217000710580916C0501C08AE0EE960FB6F89467
:10218000DEBF0FBECDBFCF91DF911F910F91FF90AA
:10219000EF90DF90CF90BF90AF909F908F907F9007
:1021A0006F905F904F903F902F900895CA80DB8092
:1021B000EC80FD80C701B6010E9432310E94E72DFC
:1021C0009B01173409F440C81D3409F0E2C97FC9E6
:1021D0001F3484F41D340CF01DCB1C340CF078CA71
:1021E00019340CF04ECA163409F410CA173409F029
:1021F0000ECB10CB143509F4A6CA153554F412359C
:1022000009F475CA13350CF08ECA103509F0FFCAEF
:1022100069CA193509F4C9CA1A3509F4DFCA18356B
:1022200009F0F5CAA9CAECE6F5E085E3DF011D92E5
:102230008A95E9F780916F0690917006A0917106DA
:10224000B09172068093740590937505A0937605FE
:10225000B09377051092850591E09093860582E012
:10226000809387059093700580918805BF01635E18
:102270007F4F0E943E1B882319F48AE00E94412868
:10228000089510920001249A259A2C9808952C986C
:1022900008951F93182F282F332727FD30958091FD
:1022A000000190E02817390771F00E944C22112399
:1022B00039F0111614F42D9801C02D9A2C9A01C0F2
:1022C0002C98109300011F910895109201013B9AE0
:1022D00043980895439808951F93182F8091010102
:1022E000181749F00E944C22113011F4439A01C092
:1022F0004398109301011F910895E0ECF0E0808174
:102300008D7F80831092C50087E68093C400E1EC46
:10231000F0E080818061808380818860808380811B
:10232000806880830895282FE09104019E2F9F5F8D
:10233000903431F490E004C080915E0584FD0FC0BC
:10234000809105019817C1F3F0E0EF5DF94F20830C
:10235000909304018091C10080628093C100089530
:102360001F920F920FB60F9211248F939F93EF93AA
:10237000FF9380910501E82FF0E0EF5DF94F908128
:102380009093C600982F9F5F903409F490E090934B
:10239000050180910401981729F48091C1008F7D77
:1023A0008093C100FF91EF919F918F910F900FBE8D
:1023B0000F901F9018959091030180910201891749
:1023C00011F4EFEF0DC0E92FF0E0EF55FA4FE08187
:1023D000892F8F5F80930301803811F410920301DD
:1023E0008E2F0895809102018093030108951F921A
:1023F0000F920FB60F9211242F933F934F935F9339
:102400006F937F938F939F93AF93BF93EF93FF93BC
:102410002091C6002132A1F0223218F42831B9F4FB
:1024200013C02F3319F02E3791F404C080915E054C
:10243000816003C080915E05826080935E0518C054
:1024400080915E058860F9CF0E94F90311C0E09188
:1024500002019E2F9F5F903809F490E08091030164
:10246000981731F0F0E0EF55FA4F20839093020176
:10247000FF91EF91BF91AF919F918F917F916F915C
:102480005F914F913F912F910F900FBE0F901F9032
:1024900018951F920F920FB60F9211242F933F930E
:1024A0004F935F936F937F938F939F93AF93BF935C
:1024B000EF93FF9386B190E0809590958770907030
:1024C000892B91F0309903C00E94F9030DC0319916
:1024D00004C080915E05886005C0329905C0809176
:1024E0005E05826080935E05FF91EF91BF91AF9191
:1024F0009F918F917F916F915F914F913F912F911C
:102500000F900FBE0F901F901895CF93DF9380917F
:102510005E05882309F457C080915E05C82FD0E07E
:10252000CE0180769070892BE9F086E080935D057E
:10253000C6FF10C08FEF0E942A2881E00E94002869
:1025400080915E058F7E80935E0580915E0584FF9D
:10255000FCCF03C08EEF0E942A2880915E058F7900
:1025600080935E05C4FF04C081E080935C052BC0AE
:10257000C0FF07C00E94992880915E058E7F8093DE
:102580005E05C3FF07C00E94011580915E05877F2D
:1025900080935E05C2FF07C00E940B1580915E0507
:1025A0008B7F80935E05C1FF0EC00E94F71480915F
:1025B000840681FF03C081E080936B0580915E05F6
:1025C0008D7F80935E05DF91CF91089580E066E076
:1025D00071E00E94AA1B882369F08091060188237C
:1025E00061F086E091E00E94E92786E091E00E9498
:1025F000E30801C08AE00E94412881E066E071E0C2
:102600000E94AA1B882321F48AE00E944128089591
:1026100080910601882351F086E091E00E94E9272D
:1026200086E091E00E94E3080E9441280895DF922D
:10263000EF92FF920F931F93DF93CF93CDB7DEB747
:1026400029970FB6F894DEBF0FBECDBF7C01FC0109
:102650008081843209F009C181E0898381818734D6
:1026600081F1883474F48432C1F0853234F48823E3
:1026700089F0833209F097C01AC0833409F093C0FF
:102680002AC08E3409F469C08835F1F1883409F024
:102690008AC04CC00E94F627F3C082E08983F7010C
:1026A0008281882309F0E6C00E94402BE9C082E0C5
:1026B0008983F7018281882309F0DCC00E94822A85
:1026C000DFC082E08983F7018281882309F0D2C0CC
:1026D0000E949629D5C082E08983F70182818823F0
:1026E00009F0C8C080915D05873021F40E94F9038C
:1026F00085E007C0882309F0BFC087E080935D05AF
:1027000084E00E940028BCC082E08983F7018281B6
:10271000882309F0AFC080915D05863009F0B0C014
:1027200083E00E94002810925D05AAC08091840673
:1027300084FD02C017E0A5C080915D05882319F0D3
:10274000863009F099C00E94B70480915C05882307
:1027500009F096C00E94E61293C082E08983F701D7
:102760008281882319F0DD24D3941EC080E0B70154
:102770000E94AA1B882329F080E0B7010E945D2AED
:1027800003C08AE00E94412881E0B7010E94AA1B91
:10279000882321F48AE00E94412872C081E0B701B9
:1027A0000E945D2A6DC0DD24C7018E010F5F1F4F9F
:1027B000B801AE014E5F5F4F0E940423892B09F4DC
:1027C0005DC09981F701E90FF11D80818D3309F01A
:1027D00051C0892F8F5F8983DD2041F1482F50E060
:1027E0002981822F90E0FC01E41BF50BEE0DFF1D0B
:1027F000D701A80FB91F8C9180838C912F5F2983FB
:10280000882371F7C7010E94E308182F8823C9F5B0
:102810006A817B818C819D810E9432310E94EC2DE6
:10282000DC01CB01B7010E949F1B2BC0C701B8017F
:10283000AE014A5F5F4F0E940423892BF9F0898122
:10284000E80EF11CF70180818823A1F46A817B8165
:102850008C819D810E94E72DDC01CB014E815F813F
:10286000688579850E94361903C0C7010E94E30874
:10287000182F07C013E005C01BE003C011E001C022
:1028800010E0812F29960FB6F894DEBF0FBECDBFA2
:10289000CF91DF911F910F91FF90EF90DF900895FE
:1028A0001F9311E044C02A3011F02D30D1F40E9462
:1028B000851280915C05882309F03FC0E0913801C2
:1028C000EE2349F0F0E0EA5FFE4F108286E091E0EF
:1028D0000E94171301C080E00E9441281092380125
:1028E00006C080913901882329F0293201F5109220
:1028F00039011DC02132D8F02F32C9F0283219F425
:102900001093390114C090913801913380F4822FD3
:102910008156E92FF0E09F5F8A3120F4EA5FFE4F95
:10292000205202C0EA5FFE4F2083909338010E943C
:10293000DB11282F8F3F09F0B6CF1F910895109219
:102940003801109239010E94FB2787B1887F87B92F
:1029500088B1876088B9ECE6F0E080818760808389
:10296000E8E6F0E0808182608083089580918406AB
:1029700082FF02C0289A01C0289880915D058330AB
:10298000F9F48091770680935D0180916E0690E066
:10299000A0E0B0E00297A109B109880F991FAA1F12
:1029A000BB1F819580935C01109259011092B20077
:1029B0008091700082608093700082E08093B1000B
:1029C00008951F920F920FB60F9211248F939F9329
:1029D0009BB1809177068C71937E892B8BB916BC45
:1029E0009F918F910F900FBE0F901F90189580911F
:1029F0005D05823029F483E080935D050E94B61462
:102A0000089580915D05833029F484E080935D050D
:102A100010926B05089580915A0190915B01892B6A
:102A2000F9F060914A0170914B0180914C019091B5
:102A30004D010E94341E81E08093580186E990E0A8
:102A4000909357018093560110924E0110924F01BE
:102A5000109250011092510182E080935D0508951B
:102A600010925D05089580E2EAE3F1E0DF011D9236
:102A70008A95E9F710925B0110925A0110925E015B
:102A80000895809170008D7F809370001092B10046
:102A9000909194069F3F21F480915E0585FF0BC0C5
:102AA000892F90E00E947D228091840682FF02C0DF
:102AB00028980895289A08958AB18C6F8AB98BB1A5
:102AC000837090917706892B8BB9209AE0E7F0E02C
:102AD00080818D7F80831092B1001092B20082E0DD
:102AE0008093B00081E48093B300EEE6F0E0808153
:102AF0008E7F808314BC15BC8081816080830E949E
:102B0000B6140E94411508951F920F920FB60F92AE
:102B10001124EF92FF920F931F932F933F934F93A4
:102B20005F936F937F938F939F93AF93BF93EF9335
:102B3000FF9380915E01882309F0CBC28BB1209175
:102B40005D01922F907E8F71982B9BB980915901D6
:102B5000882359F0109259018BB18370822B8BB965
:102B600080915C0186BD82E085BD81E080935E013D
:102B7000789480915A0190915B01892B09F082C071
:102B80000E94DC1BFC0190935B0180935A0100972B
:102B900009F453C180917706807E908189278093C4
:102BA0005D012585368547855089DA01C901B595CE
:102BB000A7959795879580933A0190933B01A093B1
:102BC0003C01B0933D0180933E0190933F01A0935F
:102BD0004001B09341018093420190934301A0933F
:102BE0004401B0934501209346013093470140933F
:102BF00048015093490120934A0130934B0140937F
:102C00004C0150934D0180915D058330D9F583A926
:102C100094A9A5A9B6A98093520190935301A093BA
:102C20005401B093550183A194A1A5A1B6A18093AD
:102C30004E0190934F01A0935001B093510186E94A
:102C400090E0909357018093560183A594A5A5A584
:102C5000B6A5281739074A075B0711F482E010C0B0
:102C6000658976898789908D21893289438954893C
:102C70000E94782D882319F41092580103C081E036
:102C80008093580120915801222309F46CC080914F
:102C900056019091570101979093570180935601E7
:102CA000892B09F060C08CE291E0909357018093EA
:102CB0005601213081F5E0915A01F0915B0187A125
:102CC00090A5A1A5B2A520914E0130914F01409150
:102CD000500150915101820F931FA41FB51F809383
:102CE0004E0190934F01A0935001B093510127A53D
:102CF00030A941A952A982179307A407B50798F1F3
:102D00001092580120934E0130934F01409350018F
:102D10005093510128C0223031F580914E0190919D
:102D20004F01A0915001B0915101E0915A01F091F1
:102D30005B0127A130A541A552A5281739074A07ED
:102D40005B072CF4821B930BA40BB50B04C088EE1D
:102D500093E0A0E0B0E080934E0190934F01A093E8
:102D60005001B0935101E0904E01F0904F0100915D
:102D700050011091510188EEE81683E0F80680E0DA
:102D8000080780E018076CF480915201909153017C
:102D9000A0915401B0915501885E9340A040B0408D
:102DA0000CC08091520190915301A0915401B091B7
:102DB00055018E199F09A00BB10B8093520190937E
:102DC0005301A0935401B0935501209152013091C9
:102DD0005301409154015091550157FF78C1E09142
:102DE0005A01F0915B0183A994A9A5A9B6A9280F5E
:102DF000391F4A1F5B1F20935201309353014093A8
:102E000054015093550180915D058430F1F4809117
:102E10005801823049F082E08093580186E990E0C1
:102E2000909357018093560187A190A5A1A5B2A5C3
:102E30008E159F05A007B10744F00E9441158091AF
:102E40005E05846080935E0542C1208120935D0110
:102E500081E08093590140913A0150913B0160918A
:102E60003C0170913D0181819281A381B481481B15
:102E7000590B6A0B7B0B40933A0150933B016093D3
:102E80003C0170933D0177FF38C0246020935D01C1
:102E90008091460190914701A0914801B09149016C
:102EA000480F591F6A1F7B1F40933A0150933B0103
:102EB00060933C0170933D0125FF0CC080915F053C
:102EC00090916005A0916105B09162050197A109FB
:102ED000B1090BC080915F0590916005A0916105DB
:102EE000B09162050196A11DB11D80935F0590937D
:102EF0006005A0936105B093620540913E01509139
:102F00003F01609140017091410185819681A781C7
:102F1000B085481B590B6A0B7B0B40933E015093C5
:102F20003F01609340017093410177FF3AC02091C7
:102F30005D01286020935D018091460190914701D9
:102F4000A0914801B0914901480F591F6A1F7B1F8A
:102F500040933E0150933F016093400170934101C3
:102F600026FF0CC08091630590916405A0916505D2
:102F7000B09166050197A109B1090BC08091630565
:102F800090916405A0916505B09166050196A11D1B
:102F9000B11D8093630590936405A0936505B0937C
:102FA0006605409142015091430160914401709146
:102FB000450181859285A385B485481B590B6A0B11
:102FC0007B0B409342015093430160934401709303
:102FD000450177FF3AC020915D01206120935D019A
:102FE0008091460190914701A0914801B09149011B
:102FF000480F591F6A1F7B1F4093420150934301A2
:10300000609344017093450127FF0CC080916705D0
:1030100090916805A0916905B0916A050197A10991
:10302000B1090BC08091670590916805A091690571
:10303000B0916A050196A11DB11D8093670590931B
:103040006805A0936905B0936A0520914A01309103
:103050004B0140914C0150914D0121503040404076
:10306000504020934A0130934B0140934C015093C0
:103070004D012115310541055105E1F080915801BF
:103080008230F1F083A594A5A5A5B6A58217930774
:10309000A407B507A8F0281739074A075B0731F4DA
:1030A00086E990E0909357018093560182E08093E7
:1030B000580106C010925B0110925A010E94CD1B6C
:1030C00080915D0190917706892780935D01109230
:1030D0005E01FF91EF91BF91AF919F918F917F9191
:1030E0006F915F914F913F912F911F910F91FF90A1
:1030F000EF900F900FBE0F901F901895F999FECF8B
:1031000092BD81BD81E08FBB80B50895F894F99997
:10311000FECF92BD81BD81E08FBB40B54627842F95
:10312000992787FD9095262F30E082239323892BC2
:1031300039F06F3F19F060BD84E006C084E104C03F
:10314000442321F060BD84E28FBBF99A78940895FE
:103150008F929F92AF92BF92CF92DF92EF92FF92A7
:103160000F93DF93CF9300D0CDB7DEB75C016B0137
:103170007A014A0100E01EC0002319F021E030E08E
:1031800008C0202F332727FD30952227330F221F19
:103190003327F60161916F01062F020F9C012F5F0B
:1031A0003F4F3A8329830E9486180894810891082A
:1031B00089819A8181149104F9F6C7018A0D9B1DBA
:1031C000602F0E9486180F900F90CF91DF910F9182
:1031D000FF90EF90DF90CF90BF90AF909F908F9037
:1031E0000895CF93DF93EC01FB019A0190E0B1E0E9
:1031F00019C0F999FECFF2BDE1BDBFBBA0B59923BF
:1032000019F081E090E008C0892F992787FD9095FB
:103210008827990F881F992731969A2F980FA9937D
:10322000215030402115310521F7460F571FF999DC
:10323000FECF52BD41BD81E08FBB80B520E030E0C4
:10324000981711F421E030E0C901DF91CF91089582
:1032500080E090E065E00E94861881E090E061E601
:1032600076E046E350E00E94A8180895EF92FF929E
:103270000F931F93CF93DF93EC017A018B01FC0135
:103280008731910540F4EC5CFF4FEE0FFF1F059076
:10329000F491E02D099486E01FC1CB01BA0120E032
:1032A00030E040E050E00E94782D181614F088E0DD
:1032B00013C1CC0FDD1FCC0FDD1FCF59D94FE882D2
:1032C000F9820A831B8305C1CB01BA0120E030E0FB
:1032D00040E450E40E94782D882314F489E0FCC077
:1032E000C801B7010E94BB300E94EC2D60936E06AE
:1032F000F0C040936F065093700660937106709310
:103300007206E7C040937306509374066093750687
:1033100070937606DEC0CB01BA010E9432310E9462
:10332000EC2D60937706D5C0CB01BA010E94BB306B
:103330000E94EC2D60939406CCC0CB01BA0120E032
:1033400030E040E752E40E94583020E030E040E7AF
:1033500052E40E94583060937C0670937D068093FF
:103360007E0690937F06B5C0DB01CA01BF778093CC
:10337000800690938106A0938206B0938306A9C02D
:10338000409378065093790660937A0670937B0693
:10339000A0C0CB01BA010E94BB300E94EC2D60930B
:1033A000960697C0CB01BA010E94BB300E94EC2D5B
:1033B000609395068EC0CB01BA0120E030E040E07A
:1033C00050E00E94782D882321F08091840681604E
:1033D00011C0809184068E7F0DC0CB01BA0120E020
:1033E00030E040E050E00E94782D882331F0809159
:1033F00084068260809384066CC0809184068D7FF1
:10340000F9CFCB01BA0120E030E040E050E00E946B
:10341000782D882321F0809184068460EBCF809101
:1034200084068B7FE7CFCB01BA0120E030E040E09B
:1034300050E00E94782D882321F0809184068860D6
:1034400003C080918406877F809384060E94BF23F7
:1034500040C0CB01BA0120E030E040E050E00E94E3
:10346000782D882321F0809184068061C3CF8091DC
:1034700084068F7EBFCFCB01BA010E9432310E94F9
:10348000EC2D6093850625C04093860650938706F1
:1034900060938806709389061CC040938A065093F7
:1034A0008B0660938C0670938D0613C0CB01BA0116
:1034B0000E94BB300E94EC2D70938F0660938E06A5
:1034C00008C04093900650939106609392067093C3
:1034D00093060E94281980E0DF91CF911F910F91F0
:1034E000FF90EF900895882309F45AC080E090E09F
:1034F000AAE7B3E48093610690936206A093630603
:10350000B09364068093650690936606A093670661
:10351000B09368068093690690936A06A0936B0641
:10352000B0936C062AE020936E0680936F0690930A
:103530007006A0937106B093720680E090E0AAEF47
:10354000B3E48093730690937406A0937506B093CA
:10355000760680E090EAACE0B7E480937C06909336
:103560007D06A0937E06B0937F068DEC9CECACECC0
:10357000BDE38093780690937906A0937A06B09382
:103580007B0680EC809377068DEC9CECACE4BDE38D
:103590008093800690938106A0938206B093830661
:1035A00082E0809384061092850680E090E0A8EC8B
:1035B000B1E48093860690938706A0938806B09323
:1035C000890680E090E0AAE7B3E480938A069093AE
:1035D0008B06A0938C06B0938D0684E690E09093C2
:1035E0008F0680938E0680E090E0A0E8BFE3809392
:1035F000900690939106A0939206B093930699E15A
:103600009093940683E080939506909396060E948B
:103610002819089580E090E00E947E18853079F4A2
:1036200081E696E061E070E046E350E00E94F11828
:1036300020E0892B09F421E081E0282712C08530A1
:1036400078F481E696E061E070E043E250E00E94A9
:10365000F118892B29F080E00E94731A21E001C043
:1036600020E0822F08959DE0899FC00111248050A1
:103670009E4F4CE050E00E94A81808950F931F93AE
:10368000CF93DF93162F072F9DE0899FE001112430
:10369000C050DE4F862F972FBE014CE050E00E94B5
:1036A000F118892B11F081E00FC0E12FF02F8CE091
:1036B000DF011D928A95E9F7CE01612F702F4CE052
:1036C00050E00E94A81880E0DF91CF911F910F91E8
:1036D0000895EF92FF921F93DF93CF93CDB7DEB79C
:1036E0002C970FB6F894DEBF0FBECDBF0E940A1B09
:1036F000882341F48AE00E94412881E00E94731AE5
:103700000E94402B10E07E010894E11CF11C812FE7
:10371000B7010E943E1B882319F48AE00E944128C9
:103720001F5F1830A1F72C960FB6F894DEBF0FBEBE
:10373000CDBFCF91DF911F91FF90EF90089593E35C
:10374000899FC001112480509D4F42E350E00E94A8
:10375000A81808950F931F93CF93DF938B0193E3E2
:10376000899FE0011124C050DD4FCB01BE0142E32F
:1037700050E00E94F118892B11F081E009C0F80196
:103780001082CE01B80142E350E00E94A81880E008
:10379000DF91CF911F910F91089590913D058091F8
:1037A0003E05981741F080913E058F5F823109F404
:1037B00080E080933E05089590913D0580913E05FF
:1037C000981719F420E030E008C090913E0587E397
:1037D000989F90011124215A3E4FC901089590915C
:1037E0003E0520E080913F05981709F421E0822FE3
:1037F0000895EF92FF920F931F936093400570938B
:1038000041058093420590934305209344053093EE
:1038100045054093460550934705E0924805F092D0
:10382000490500934A0510934B051F910F91FF9096
:10383000EF9008952F923F924F925F926F927F92F6
:103840008F929F92AF92BF92CF92DF92EF92FF92B0
:103850000F931F93DF93CF9300D000D0CDB7DEB787
:103860001C016A017B0148015901CB01BA0124EE18
:1038700038E34EE552E40E9458300E94652D0E94C4
:10388000EC2DF10163A374A385A396A365857685CA
:10389000878590890E941A2E2B013C0120917C067D
:1038A00030917D0640917E0650917F06CA01B90194
:1038B0000E949F2CF101258D368D478D50A10E94CD
:1038C00058309B01AC01C301B2010E947F2D698376
:1038D0007A838B839C83C501B401A50194010E9466
:1038E00058304B015C01C701B601A70196010E9447
:1038F0005830A50194010E949E2C9B01AC01698166
:103900007A818B819C810E9458309B01AC01C3015C
:10391000B2010E949F2C20E030E040E05FE30E9473
:1039200058300E94652D0E94E72D7B018C011616F0
:1039300017061806190634F0F10113A614A615A6E9
:1039400016A639C0F1012189328943895489CA01F7
:10395000B9010E945830A50194010E949E2C9B0140
:10396000AC0169817A818B819C810E9458300E94D0
:10397000652D0E94EC2DF10163A774A785A796A77A
:10398000E616F7060807190720F4E3A6F4A605A72C
:1039900016A7F101258536854785508983A594A50D
:1039A000A5A5B6A5281739074A075B0720F423A762
:1039B00034A745A756A70F900F900F900F90CF9167
:1039C000DF911F910F91FF90EF90DF90CF90BF900C
:1039D000AF909F908F907F906F905F904F903F90AF
:1039E0002F9008953F924F925F926F927F928F92A5
:1039F0009F92AF92BF92CF92DF92EF92FF920F937E
:103A00001F93CF93DF9390903D0540907C0650909C
:103A10007D0660907E0670907F0600E010E0C0E0BA
:103A2000D0E03324339427E3822E6DC0992011F423
:103A300092E1992E9A94209709F45EC00115110520
:103A400009F45AC0D98CCA8CBB8CAC8C6D897E8928
:103A50008F89988D2D2D3C2D4B2D5A2D0E94782D20
:103A6000882309F449C08AA18823E9F5F801E5888B
:103A7000F6880789108D6D2D7C2D8B2D9A2DA80130
:103A800097010E94862F181674F5C801B701A80186
:103A900097010E9458307B018C01C301B201A30140
:103AA00092010E949F2C2D8D3E8D4F8D58A10E941A
:103AB00058309B01AC01C801B7010E949F2C0E94A5
:103AC000E530162F072FF82EE92E6D2D7C2D8B2D2E
:103AD0009A2D212F302F4F2D5E2D0E94782D87FD9E
:103AE00002C0680157018D2D9C2DAB2DBA2D8D8BF9
:103AF0009E8BAF8BB88F39A2989CC00111248E0188
:103B0000EC01C15ADE4F80913E05981609F08ECF28
:103B100070903E05C0E0D0E087E3582E66246394A1
:103B200080C0759C600111248FE591E0C80ED91EFC
:103B3000209709F470C08AA1882309F058C0ED8845
:103B4000FE880F89188DF601B588A6889788808C25
:103B5000C801B7012B2D3A2D492D582D0E94782DE3
:103B600088230CF044C0C801B701A80197010E9446
:103B700058307B018C0120917C0630917D0640916C
:103B80007E0650917F06CA01B9010E949F2C2D8D9F
:103B90003E8D4F8D58A10E9458309B01AC01C80149
:103BA000B7010E949F2C0E94E5307B018C016B2D98
:103BB0007A2D892D982D9701A8010E94782D8823B0
:103BC00024F4EB2CFA2C092D182D6B2D7A2D892D30
:103BD000982D9701A8010E94782D882341F0C701F4
:103BE000D801F601858B968BA78BB08F61A289A136
:103BF000882321F4F60181A1882369F04D895E892B
:103C00006F89788DF601058916892789308DCE0157
:103C10000E941A1C19A27394F2E17F1609F477240A
:103C2000E60180913D05781609F07BCF4D895E89CC
:103C30006F89788DCE0100E010E020E030E00E9436
:103C40001A1C19A2DF91CF911F910F91FF90EF9055
:103C5000DF90CF90BF90AF909F908F907F906F90AC
:103C60005F904F903F900895AF92BF92CF92DF92B6
:103C7000EF92FF920F931F93CF93DF935B016C0141
:103C800090913E0587E3989FE0011124C15ADE4FD1
:103C9000C601B5010E941A2E2D8D3E8D4F8D58A163
:103CA0000E9458307B018C016D857E858F859889B7
:103CB0000E941A2E9B01AC01C801B7010E947F2D02
:103CC0006D8F7E8F8F8F98A3AD86BE86CF86D88A64
:103CD00080E090E0A0E0B0E08D8B9E8BAF8BB88F42
:103CE000898F9A8FAB8FBC8F1AA281E089A30E9423
:103CF000F21CDF91CF911F910F91FF90EF90DF9019
:103D0000CF90BF90AF9008952F923F924F925F92C5
:103D10006F927F928F929F92AF92BF92CF92DF92DB
:103D2000EF92FF920F931F93DF93CF93CDB7DEB740
:103D3000EF970FB6F894DEBF0FBECDBF29013A0151
:103D4000AFA6B8AAC9AADAAA8BAA30913D0527E383
:103D5000329FA0011124415A5E4F5A8F498F209102
:103D600061063091620640916306509164062BA76C
:103D70003CA74DA75EA70E9458300E9428306CAB2C
:103D80007DAB8EAB9FAB8091650690916606A0914E
:103D90006706B09168068FA398A7A9A7BAA7C30121
:103DA000B2012FA138A549A55AA50E9458300E94FA
:103DB000283068AF79AF8AAF9BAFA0906906B0900A
:103DC0006A06C0906B06D0906C06C801B701A601C8
:103DD00095010E9458300E9428306CAF7DAF8EAFA5
:103DE0009FAFE0904005F090410500914205109191
:103DF0004305EBA2FCA20DA31EA32CA93DA94EA92D
:103E00005FA92E193F09400B510BA98DBA8D119650
:103E10002D933D934D935C93149757FF0DC08827C6
:103E20009927DC01821B930BA40BB50BE98DFA8D4E
:103E300081839283A383B483E0904405F090450589
:103E40000091460510914705EF8EF8A209A31AA329
:103E500028AD39AD4AAD5BAD2E193F09400B510B72
:103E6000A98DBA8D15962D933D934D935C9318971C
:103E700057FF0DC088279927DC01821B930BA40BE9
:103E8000B50BE98DFA8D85839683A783B087E09083
:103E90004805F090490500914A0510914B05EB8EBD
:103EA000FC8E0D8F1E8F2CAD3DAD4EAD5FAD2E192E
:103EB0003F09400B510B57FF07C050954095309577
:103EC00021953F4F4F4F5F4FA98DBA8D19962D9376
:103ED0003D934D935C931C971596ED90FD900D913D
:103EE0001C911897FD0181819281A381B4818E1567
:103EF0009F05A007B10710F4D801C70182179307E7
:103F0000A407B50710F4DA01C901E98DFA8D858798
:103F10009687A787B08B0097A105B10509F4A3C2C6
:103F200061817281838194810E94182E2BA53CA50A
:103F30004DA55EA50E947F2D1B012C01A98DBA8D78
:103F400015966D917D918D919C9118970E94182ED8
:103F50002FA138A549A55AA50E947F2D3B014C01F0
:103F6000E98DFA8D61857285838594850E94182E6E
:103F7000A60195010E947F2D5B016C01C201B10178
:103F8000A20191010E9458307B018C01C401B30150
:103F9000A40193010E9458309B01AC01C801B701F4
:103FA0000E949F2C7B018C01C601B501A6019501E1
:103FB0000E9458309B01AC01C801B7010E949F2CA0
:103FC0000E94E5309B01AC01A98DBA8D5D966D9381
:103FD0007D938D939C93909760E070E080E89FE3E1
:103FE0000E947F2D7B018C01C201B101A8019701C4
:103FF0000E9458301B012C016D877E878F87988B1C
:10400000C401B301A80197010E9458303B014C0143
:10401000698B7A8B8B8B9C8BC601B501A8019701AC
:104020000E9458309B01AC016D8B7E8B8F8B988FDB
:10403000E98DFA8D1082ECA8FDA80EA91FA98BA10D
:104040009CA1ADA1BEA1E816F9060A071B074CF416
:1040500080E28083D201C101B0588D879E87AF87EF
:10406000B88BE8ACF9AC0AAD1BAD8F8D98A1A9A1B6
:10407000BAA1E816F9060A071B0764F4A98DBA8DE0
:104080008C9180648C93D401C301B058898B9A8B36
:10409000AB8BBC8BECACFDAC0EAD1FAD8B8D9C8D9A
:1040A000AD8DBE8DE816F9060A071B0764F4A98DCD
:1040B000BA8D8C9180688C93DA01C901B0588D8BD0
:1040C0009E8BAF8BB88FBBA9BB2381F0E98DFA8D96
:1040D000658D768D878D90A12FA538A949A95AA9FC
:1040E0000E947F2D6FA778AB89AB9AABEFA4F8A89D
:1040F00009A91AA9A98DBA8D5196ED92FD920D9339
:104100001C93549760907C0670907D0680907E068C
:1041100090907F06C401B30126E234EB47E15CE3F3
:104120000E9458300E94652D0E94E72DE98DFA8D7E
:1041300067A370A781A792A7C801B70124EE38E34F
:104140004EE552E40E9458300E94652D0E94EC2DED
:10415000A98DBA8D9F966D937D938D939C93D297E5
:104160005D966D917D918D919C91909720E23CEBB5
:104170004EEB5CE40E9458307B018C01E98DFA8D96
:1041800065857685878590890E941A2E9B01AC01F2
:10419000C801B7010E947F2D0E94652D0E94EC2D61
:1041A000A98DBA8DD3966D937D938D939C93D6975D
:1041B00090913D0580913E05981709F4B3C0209079
:1041C00058053090590540905A0550905B05B10153
:1041D000C20120E030E040E050E00E94862F181637
:1041E0000CF0A0C060914C0570914D0580914E057A
:1041F00090914F0590582D853E854F8558890E9496
:1042000058307B018C01609150057091510580916F
:1042100052059091530529893A894B895C890E94FE
:1042200058309B01AC01C801B7010E949E2C7B0154
:104230008C016091540570915505809156059091BF
:1042400057052D893E894F89588D0E9458309B0112
:10425000AC01C801B7010E949E2C7B018C0123E3B5
:1042600033E343E75FE30E94782D88230CF05AC0C4
:10427000B101C2012FA538A949A95AA90E94782DD8
:1042800087FD06C08FA598A9A9A9BAA91C012D016F
:10429000C801B70123E333E343E75FEB0E94862FB6
:1042A00018160CF044C060E070E080E89FE3A801BD
:1042B00097010E949E2C20E030E040E05FE30E94E6
:1042C00058300E94E5305B016C01C401B3012091BC
:1042D00080063091810640918206509183060E94AB
:1042E0005830A60195010E9458307B018C0160E096
:1042F00070E080E89FE3A60195010E949E2C9B013F
:10430000AC01C801B7010E947F2D0E94E5307B01FE
:104310008C01B101C2019701A8010E94782D87FD8F
:1043200006C007C0EE24FF2400E010E002C07101C7
:104330008201C701D801E98DFA8D818F928FA38FF9
:10434000B48FC401B301A40193010E949F2CA98DD5
:10435000BA8D5D962D913D914D915C9190970E9403
:10436000583020E030E040E050E00E949F2C0E9456
:10437000E530D62EC72EB82EA92EB701C8012D2D97
:104380003C2D4B2D5A2D0E94782D87FD04C0ED2C1D
:10439000FC2C0B2D1A2DC701D801E98DFA8D858BC8
:1043A000968BA78BB08F61897289838994892D2D13
:1043B0003C2D4B2D5A2D0E94782D181634F081E09B
:1043C000A98DBA8D92968C9303C0E98DFA8D12A2B5
:1043D00081E0A98DBA8D91968C93ECACFDAC0EADBD
:1043E0001FADE986FA860B871C8708AD19AD2AAD8B
:1043F0003BAD0D831E832F8338872CA93DA94EA981
:104400005FA929833A834B835C83ACE4B5E0FE016A
:104410003D968CE001900D928150E1F7E98DFA8D87
:1044200081899289A389B48980935805909359050D
:10443000A0935A05B0935B0580913F0580933D059D
:1044400080913D058F5F823109F480E080933F05C4
:10445000A0E4B5E0FE0131968CE001900D92815010
:10446000E1F70E94F21CEF960FB6F894DEBF0FBE84
:10447000CDBFCF91DF911F910F91FF90EF90DF9013
:10448000CF90BF90AF909F908F907F906F905F90F4
:104490004F903F902F9008951F9317E306C00E94FE
:1044A000851280915C05882391F490913D0580915F
:1044B0003E05981741F080913E05819FC00111246F
:1044C000815A9E4F61F780915D05833041F31F91C2
:1044D000089580913D0580933E0580913D058F5F55
:1044E000823109F480E080933F058CE1E0E4F5E05F
:1044F000DF011D928A95E9F7089520EA3FE004C0A4
:10450000F9013197F1F701970097D1F708951F93BB
:10451000A0EABFE040E951E015E335E031C06A3080
:1045200071058105910540F4232F2A95F1F761501B
:1045300070408040904024C064367105810591052B
:1045400040F4212F2A95F1F76A5070408040904046
:1045500017C0683E23E0720720E0820720E0920740
:1045600040F4FA013197F1F7645670408040904072
:1045700007C0FD013197F1F7685E734080409040BD
:10458000611571058105910551F61F910895EF920E
:10459000FF920F931F9360915F057091600580916A
:1045A0006105909162052091630530916405409109
:1045B000650550916605E0906705F09068050091EB
:1045C000690510916A050E94F91B60915F05709161
:1045D000600580916105909162052091630530919D
:1045E00064054091650550916605E0906705F0907F
:1045F00068050091690510916A050E9490081F9155
:104600000F91FF90EF9008956F927F928F929F92FB
:10461000AF92BF92CF92DF92EF92FF920F931F93D0
:10462000CF93DF934C013B015A01FB018081F401E0
:10463000E80FF11DEF0189918D3229F481812196D6
:10464000CC24C39405C08B3211F481812196CC24F3
:1046500020E030E040E050E0DD24E0E070E0682F52
:1046600060536A30F8F4EF5FE930C0F47111DA9406
:10467000DA01C901F2E0880F991FAA1FBB1FFA9542
:10468000D1F7280F391F4A1F5B1F220F331F441F0A
:10469000551F260F311D411D511D09C0772339F4C7
:1046A000D39405C06E3F29F4772319F471E0899102
:1046B000D6CFEE2319F420E030E051C0CA01B90191
:1046C0000E94182E7B018C0120E030E040E050E099
:1046D0000E94782D882369F42BC0C801B7012AE015
:1046E00037ED43E25CE30E9458307B018C01F2E03D
:1046F000DF0E8FEFD8168CF3D81659F4C801B70126
:104700002DEC3CEC4CEC5DE30E9458307B018C01BD
:104710000FC0DD2069F0C801B70120E030E040E2C1
:1047200051E40E9458307B018C01DA941D149CF3F3
:10473000CC2049F0D801C701B058F501808391839E
:10474000A283B38305C0F501E082F1820283138363
:10475000882D80958C0FF301808321E030E0C90122
:10476000DF91CF911F910F91FF90EF90DF90CF904D
:10477000BF90AF909F908F907F906F90089584B17D
:10478000817F84B985B18E6085B98091840683FF6D
:1047900009C080916B008E6080936B0080916800EF
:1047A000816008C080916B00817F80936B00809155
:1047B00068008E7F8093680008952F923F924F92F9
:1047C0005F926F927F928F929F92AF92BF92CF92A1
:1047D000DF92EF92FF920F931F93DF93CF93CDB7AA
:1047E000DEB7A9970FB6F894DEBF0FBECDBF382E47
:1047F000562E49A738014901FE0131968CE0DF01B0
:104800001D928A95E9F7032D30FC02C010E00FC01D
:1048100060916106709162068091630690916406D2
:104820000E94283069837A838B839C8311E001FF87
:104830000FC01F5F609165067091660680916706E4
:10484000909168060E9428306D837E838F839887BD
:1048500002FF0FC01F5F6091690670916A06809128
:104860006B0690916C060E94283069877A878B8747
:104870009C8789859A85AB85BC852D813E814F813A
:1048800058852DA33EA34FA358A7281739074A07D9
:104890005B0720F48DA39EA3AFA3B8A789819A815B
:1048A000AB81BC814DA15EA16FA178A548175907C6
:1048B0006A077B0720F48DA39EA3AFA3B8A7612F3F
:1048C00070E080E090E00E94182E0E94E5305B01CD
:1048D0006C016DA17EA18FA198A50E94182EA60142
:1048E00095010E947F2D7B018C0120917C063091E7
:1048F0007D0640917E0650917F060E94583020E050
:1049000030E84BEB55E40E947F2D0E94652D0E94FC
:10491000EC2D69A37AA38BA39CA3C401B301A601C8
:1049200095010E9458309B01AC01C801B7010E945B
:1049300058309B01AC0160EC71EE84E69CE40E946F
:104940007F2D0E9428307B018C0158EFE51654E240
:10495000F50651E0050750E0150718F45701680106
:1049600007C038EFA32E34E2B32E31E0C32ED12C92
:104970004090850660EE46228091770648265520B5
:1049800011F480EE48268DA19EA1AFA1B8A5B695E1
:10499000A79597958795662477244301681A790A25
:1049A0008A0A9B0A80916E06A6019501281B31098F
:1049B000410951092D8B3E8B4F8B588F6D8E7E8E0A
:1049C0008F8E98A2698E7A8E8B8E9C8E198A1A8A07
:1049D0001B8A1C8A48E853E160E070E04D875E87DF
:1049E0006F87788B84E0282E242423B159A5552382
:1049F00011F06EE0262730FE1DC089819A81AB81BF
:104A0000BC81680E791E8A1E9B1E1614170418049A
:104A1000190484F421FF02C0522C03C07EEF372218
:104A2000542C8DA19EA1AFA1B8A5681A790A8A0A53
:104A30009B0A01C0542C31FE2CC08D819E81AF8118
:104A4000B8854D8D5E8D6F8D78A1480F591F6A1FF7
:104A50007B1F4D8F5E8F6F8F78A314161506160679
:104A60001706BCF422FF03C058E0552602C06DEFC4
:104A700036228D8D9E8DAF8DB8A14DA15EA16FA107
:104A800078A5841B950BA60BB70B8D8F9E8FAF8FD0
:104A9000B8A332FE2CC089859A85AB85BC85498D2B
:104AA0005A8D6B8D7C8D480F591F6A1F7B1F498F54
:104AB0005A8F6B8F7C8F1416150616061706BCF4DA
:104AC00023FF03C050E1552602C06BEF3622898DCB
:104AD0009A8DAB8DBC8D2DA13EA14FA158A5821BF7
:104AE000930BA40BB50B898F9A8FAB8FBC8F0E9451
:104AF0008512332009F46AC080915C05882309F08F
:104B000065C08BB13CE15322837E582A5BB860912B
:104B10006E0670E080E090E00E9487224BB86D89BD
:104B20007E898F89988D0E948722EA14FB040C05E8
:104B30001D0508F05ACF4D855E856F8578894A0D31
:104B40005B1D6C1D7D1D4D875E876F87788B4131A6
:104B500087E2580780E0680780E0780708F445CFCF
:104B600040515742604070404D875E876F87788B19
:104B700029893A894B895C8969A17AA18BA19CA179
:104B8000260F371F481F591F298B3A8B4B8B5C8B85
:104B900060E077E883E993E00E945131C901DA01CE
:104BA0005C016D01AE14BF04C006D10610F45701BC
:104BB000680180916E06A6019501281B3109410903
:104BC00051092D8B3E8B4F8B588F0FCFA9960FB667
:104BD000F894DEBF0FBECDBFCF91DF911F910F9133
:104BE000FF90EF90DF90CF90BF90AF909F908F900D
:104BF0007F906F905F904F903F902F900895FF921D
:104C00000F931F930E94B61400918A0610918B0691
:104C100020918C0630918D0684E061E040E00E9496
:104C2000DD2300918A0610918B0620918C0630912D
:104C30008D0683E061E040E00E94DD2380918E06D6
:104C400090918F060E947D2242E0F42EFA9400910A
:104C5000860610918706209188063091890687E0A4
:104C600060E041E00E94DD2380918E0690918F06E6
:104C70000E947D2281E0F816A1F400918606109131
:104C80008706209188063091890687E061E040E040
:104C90000E94DD2380918E0690918F060E947D22D6
:104CA000D5CFFF2099F60E9441151F910F91FF90DB
:104CB00008951F920F920FB60F9211242F933F93D6
:104CC0004F935F936F937F938F939F93AF93BF9314
:104CD000EF93FF9380915D05863059F080915E05DA
:104CE00085FD07C00E94F90380915E058064809372
:104CF0005E05FF91EF91BF91AF919F918F917F9151
:104D00006F915F914F913F912F910F900FBE0F9038
:104D10001F9018958F929F92AF92BF92CF92DF9281
:104D2000EF92FF920F931F93DF93CF93CDB7DEB730
:104D30002A970FB6F894DEBF0FBECDBF7B018C0162
:104D400020E030E040E050E00E94782D88233CF4E1
:104D50008DE20E94931117FB109517F91095A09002
:104D60009506DA2C0CC0C801B70120E030E048EC11
:104D700052E40E9458307B018C018EEFD80EE1E0A6
:104D8000ED1588F3A0FE0AC0C801B70120E030E0AD
:104D900040E251E40E9458307B018C01C801B70108
:104DA00020E030E040E05FE30E949F2C0E94E72D6E
:104DB0006B017C019E012F5F3F4FF901EA0DF11D50
:104DC0008EE28083BB2449011EC0BA1409F4B39457
:104DD00084010B0D111DC701B6012AE030E040E04F
:104DE00050E00E945131605DF8016083B394C701C7
:104DF000B6012AE030E040E050E00E945131C901A4
:104E0000DA016C017D01C114D104E104F104E9F679
:104E100006C0FC01EB0DF11D2083B39403C0CE014D
:104E2000019620E3BA14A8F3BA1489F48B2D8F5F8E
:104E3000FE01E80FF11D90E39183B82EB39407C0F3
:104E4000FE01EB0DF11D80810E949311BA94BB20ED
:104E5000B9F72A960FB6F894DEBF0FBECDBFCF913B
:104E6000DF911F910F91FF90EF90DF90CF90BF9057
:104E7000AF909F908F9008958F929F92BF92CF9204
:104E8000DF92EF92FF920F931F93DF93CF93CDB7F3
:104E9000DEB72A970FB6F894DEBF0FBECDBF7B01F9
:104EA0008C0197FF0BC08DE20E9493111095009525
:104EB000F094E094E11CF11C011D111D67017801C3
:104EC000C114D104E104F10421F480E30E949311A0
:104ED0002FC0BB244E010894811C911C84010B0D32
:104EE000111DC701B6012AE030E040E050E00E9409
:104EF0005131605DF8016083B394C701B6012AE0C7
:104F000030E040E050E00E945131C901DA016C010B
:104F10007D01C114D104E104F10401F707C0FE01D1
:104F2000EB0DF11D80810E949311BA94BB20B9F75B
:104F30002A960FB6F894DEBF0FBECDBFCF91DF919A
:104F40001F910F91FF90EF90DF90CF90BF909F90B7
:104F50008F9008950F931F93DF93CF93CDB7DEB754
:104F600028970FB6F894DEBF0FBECDBF982FFE0175
:104F700031969E01275F3F4F892F817081939695CF
:104F8000E217F307C9F78E01085F1F4FF801808110
:104F9000805D0E949311015010400C171D07B1F75E
:104FA00028960FB6F894DEBF0FBECDBFCF91DF912C
:104FB0001F910F910895CF93DF93EC0102C00E94DF
:104FC0009311FE01219684918823C9F7DF91CF9137
:104FD0000895CF93DF93EC0103C021960E949311B3
:104FE00088818823D1F7DF91CF9108958AE594E0F5
:104FF0000E94DB27089588E895E00E94DB2708954A
:105000001F93182F82EF95E00E94DB27133091F059
:10501000143028F4113041F01230B1F408C01430CB
:1050200061F0153089F40CC080EE95E00BC08CEC7B
:1050300095E008C08AEB95E005C082EB95E002C0E0
:1050400089EA95E00E94DB2785EA95E00E94DB274C
:105050001F9108951F93182F8CE196E00E94DB2783
:105060001E3F29F01F3F39F481E196E002C08EEF28
:1050700095E00E94DB2784EF95E00E94DB271F91DB
:1050800008951F93182F882319F48DE097E04DC0E1
:1050900085E097E00E94DB27163079F1173070F435
:1050A000133011F1143028F41130C1F01230D9F559
:1050B00018C01430E1F01530B1F51CC0193031F1D1
:1050C0001A3028F41730E1F0183069F51CC01B3095
:1050D00019F11B30F0F01C3031F521C083EF96E060
:1050E00020C08BED96E01DC085EC96E01AC086EBE3
:1050F00096E017C080EA96E014C08EE896E011C0F2
:105100008DE796E00EC081E796E00BC082E696E060
:1051100008C081E496E005C082E396E002C087E221
:1051200096E00E94DB2784E296E00E94DB271F9135
:105130000895AF92BF92CF92DF92EF92FF920F93BA
:105140001F93DF93CF93CDB7DEB768970FB6F89470
:10515000DEBF0FBECDBFDE011196EFE5F5E08CE0BE
:1051600001900D928150E1F780915D058430C9F086
:10517000853038F4823079F0833080F4882341F030
:105180001DC08630A1F0863078F08730B9F412C0A7
:105190008CE191E011C085E191E00EC080E191E0E9
:1051A0000BC08AE091E008C084E091E005C08DEF7B
:1051B00090E002C086EF90E00E94DB278FEE90E047
:1051C0000E94DB278DE0E82EF12CEC0EFD1E67011E
:1051D00000E010E05E010894A11CB11CF501E00F95
:1051E000F11F60817181828193810E941A2EF801E2
:1051F000EF59F94F20813181428153810E947F2DE7
:105200009B01AC01F601608371838283938380915B
:10521000840680FF0DC0CA01B9012BE832E441E2E7
:105220005DE30E945830F60160837183828393832B
:10523000F60161917191819191916F010E948A268D
:105240008DEE90E00E94DB270C5F1F4F0C301105A4
:1052500029F687EE90E00E94DB2709E815E0DD24BF
:105260008091840680FF1BC0F8016081718182817A
:10527000938124853585468557850E949F2C2BE890
:1052800032E441E25DEB0E9458309B01AC01F70132
:1052900060817181828193810E949F2C14C0F801EA
:1052A000608171818281938124853585468557850A
:1052B0000E949F2C9B01AC01F7016081718182816A
:1052C00093810E949E2CF701608371838283938374
:1052D000F70160817181828193810E948A26F2E0C8
:1052E000DF1621F085EE90E00E94DB27D39484E066
:1052F00090E0E80EF91E0C5F1F4F93E0D91609F0FD
:10530000AFCF81EE90E00E94DB2768960FB6F8944D
:10531000DEBF0FBECDBFCF91DF911F910F91FF90E8
:10532000EF90DF90CF90BF90AF90089580916D0582
:10533000823091F0833028F4882341F08130B1F439
:1053400008C0833061F0843089F40CC085E991E0B5
:105350000BC081E991E008C08DE891E005C089E8C3
:1053600091E002C084E891E00E94DB2781E891E0AF
:105370000E94DB276091880570E06A5C7F4F882778
:1053800077FD8095982F0E943C2780918505882382
:1053900051F480918605813019F48CE791E005C0C5
:1053A00087E791E002C082E791E00E94DB278091CD
:1053B0006F05882319F08DE691E002C088E691E040
:1053C0000E94DB2780917005882319F083E691E025
:1053D00002C08EE591E00E94DB2780916E05882354
:1053E00019F089E591E002C084E591E00E94DB2795
:1053F00080917105813041F0813018F0823059F48C
:1054000006C080E591E005C08CE491E002C088E42C
:1054100091E00E94DB2780917205882359F081304A
:1054200019F08F3F59F403C084E491E005C080E493
:1054300091E002C08CE391E00E94DB27809173052C
:10544000882319F0813041F403C088E391E002C061
:1054500084E391E00E94DB2781E391E00E94DB2757
:105460006091840570E080E090E00E943C278EE22D
:1054700091E00E94DB2780916F05882379F060918D
:1054800074057091750580917605909177052BE8EC
:1054900032E441E25DE30E94583008C06091740537
:1054A0007091750580917605909177050E948A2606
:1054B0008AE291E00E94DB270895CF92DF92EF927B
:1054C000FF920F931F93E82E6B0187E291E00E94F9
:1054D000DB27FF2400E010E0C801B7010E943C2751
:1054E00085E291E00E94DB27C6010E94E92782E263
:1054F00091E00E94DB271F910F91FF90EF90DF90CA
:10550000CF900895CF92DF92EF92FF920F931F9367
:10551000DF93CF93CDB7DEB72C970FB6F894DEBFED
:105520000FBECDBFFF246E010894C11CD11C8F2D6E
:10553000B6010E943E1B882321F48AE00E94412884
:1055400090C08BEC91E00E94DB2783E0F816E9F035
:105550008F1530F0E1E0FE1691F0EF1598F00CC0D9
:10556000F5E0FF16C1F0FF1698F086E0F816B1F0EE
:10557000E7E0FE16D1F415C087EC91E014C083EC8F
:1055800091E011C08FEB91E00EC08BEB91E00BC06E
:1055900087EB91E008C083EB91E005C08FEA91E0D2
:1055A00002C08BEA91E00E94DB278601EE24809105
:1055B000840680FF0CC0F801608171818281938133
:1055C0002BE832E441E25DE30E94583005C0F80167
:1055D00060817181828193810E948A26F2E0EF16B8
:1055E00019F089EA91E002C085EA91E00E94DB2788
:1055F000E3940C5F1F4F83E0E816C9F6F394E8E0EC
:10560000FE1609F094CF8FE991E00E94DB2705E9AF
:1056100015E0FF248091840680FF0CC0F8016081B2
:105620007181828193812BE832E441E25DE30E9443
:10563000583005C0F80160817181828193810E9498
:105640008A26F2E0FF1619F08DE991E002C089E99F
:1056500091E00E94DB27F3940C5F1F4F83E0F81664
:10566000C9F62C960FB6F894DEBF0FBECDBFCF9112
:10567000DF911F910F91FF90EF90DF90CF900895F1
:1056800086E594E00E94DB276091610670916206D6
:1056900080916306909164060E948A2683E494E0D8
:1056A0000E94DB276091650670916606809167060F
:1056B000909168060E948A2680E394E00E94DB278E
:1056C0006091690670916A0680916B0690916C06F4
:1056D0000E948A268DE194E00E94DB2760916E068D
:1056E00070E080E090E00E943C2784E094E00E941B
:1056F000DB2760916F067091700680917106909122
:1057000072060E948A2687EE93E00E94DB27609152
:1057100073067091740680917506909176060E94CA
:105720008A268AEC93E00E94DB276091770670E07E
:1057300080E090E00E943C278CEA93E00E94DB2707
:10574000809177060E94AA2785EA93E00E94DB27D2
:105750006091940670E080E090E00E943C2787E82A
:1057600093E00E94DB2760917C0670917D0680911A
:105770007E0690917F0620E030E041E655E40E94ED
:105780007F2D0E948A2688E693E00E94DB276091A5
:1057900080067091810680918206909183060E9416
:1057A0008A2688E493E00E94DB2760917806709156
:1057B000790680917A0690917B060E948A268FE274
:1057C00093E00E94DB276091960670E080E090E015
:1057D0000E943C2780E193E00E94DB2760919506C0
:1057E00070E080E090E00E943C2787EF92E00E940A
:1057F000DB276091840670E080E090E0617070705B
:10580000807090700E943C278AED92E00E94DB2716
:105810006091840670E07695679580E090E0617015
:105820007070807090700E943C2780EC92E00E9423
:10583000DB276091840670E076956795769567958D
:1058400080E090E061707070807090700E943C27E2
:105850008EE992E00E94DB276091840670E023E0ED
:10586000769567952A95E1F780E090E06170707019
:10587000807090700E943C2783E892E00E94DB27B2
:105880006091840670E094E0769567959A95E1F7CB
:1058900080E090E061707070807090700E943C2792
:1058A00087E692E00E94DB276091850670E080E049
:1058B00090E00E943C2788E492E00E94DB278091E0
:1058C00085060E94AA2780E492E00E94DB2760916F
:1058D00086067091870680918806909189060E94BD
:1058E0008A2683E292E00E94DB2760918A0670910B
:1058F0008B0680918C0690918D060E948A2686E008
:1059000092E00E94DB2760918E0670918F0680E006
:1059100090E00E943C2787EE91E00E94DB27609197
:1059200090067091910680919206909193060E9444
:105930008A268EEC91E00E94DB2708955058BB2701
:10594000AA270ED081C241D230F046D220F031F4E5
:105950009F3F11F41EF411C20EF4E095E7FBDCC189
:10596000E92F94D280F3BA1762077307840795076B
:1059700018F071F49EF5C3C20EF4E0950B2EBA2F09
:10598000A02D0B01B90190010C01CA01A001112445
:10599000FF27591B99F0593F50F4503E68F11A16F1
:1059A000F040A22F232F342F4427585FF3CF469582
:1059B00037952795A795F0405395C9F77EF41F16A4
:1059C000BA0B620B730B840BBAF09150A1F0FF0F6E
:1059D000BB1F661F771F881FC2F70EC0BA0F621F5A
:1059E000731F841F48F4879577956795B795F7954A
:1059F0009E3F08F0B3CF9395880F08F09927EE0FDC
:105A0000979587950895E1D158F080E891E009F4E1
:105A10009EEFE2D128F040E851E059F45EEF09C072
:105A2000ACC16DC2E92FE07831D268F3092E052AA6
:105A3000C1F3261737074807590738F00E2E07F825
:105A4000E02569F0E025E0640AC0EF6307F8009400
:105A500007FADB01B9019D01DC01CA01AD01EF9339
:105A60005DD0F2D10AD05F91552331F02BED3FE0AC
:105A700049E450FD49EC63CF0895DF93DD27B92F4A
:105A8000BF7740E85FE31616170648075B0710F478
:105A9000D92FA1D29F938F937F936F93E0D3E6E9A1
:105AA000F0E06ED1D1D12F913F914F915F910CD306
:105AB000DD2349F09058A2EA2AED3FE049EC5FE38C
:105AC000D0785D274DDFDF91BFC102D280F09F37D4
:105AD00040F491110EF414C260E070E080E89FE39E
:105AE000089526F01B16611D711D811D1BC135C156
:105AF000EFD008F481E0089577D1E395B6C10CD0DA
:105B0000A3C16AD140F061D130F021F45F3F19F0B8
:105B100003C15111F5C131C1B9D198F39923C9F32A
:105B20005523B1F3951B550BBB27AA2762177307A3
:105B3000840738F09F5F5F4F220F331F441FAA1F57
:105B4000A9F333D00E2E3AF0E0E830D09150504017
:105B5000E695001CCAF729D0FE2F27D0660F771FC5
:105B6000881FBB1F261737074807AB07B0E809F0A7
:105B7000BB0B802DBF01FF2793585F4F2AF09E3F3C
:105B8000510568F0C9C0BCC15F3FECF3983EDCF33F
:105B9000869577956795B795F7959F5FC9F7880FB5
:105BA000911D9695879597F90895E1E0660F771F07
:105BB000881FBB1F621773078407BA0720F0621B98
:105BC000730B840BBA0BEE1F88F7E095089504D091
:105BD0006894B11195C1089561D188F09F5790F0F4
:105BE000B92F9927B751A0F0D1F0660F771F881F02
:105BF000991F1AF0BA95C9F712C0B13081F07FD160
:105C0000B1E008957CC1672F782F8827B85F39F0FD
:105C1000B93FCCF3869577956795B395D9F73EF460
:105C200090958095709561957F4F8F4F9F4F089508
:105C3000E89409C097FB3EF4909580957095619526
:105C40007F4F8F4F9F4F9923A9F0F92F96E9BB27DC
:105C50009395F695879577956795B795F111F8CF58
:105C6000FAF4BB0F11F460FF1BC06F5F7F4F8F4FC3
:105C70009F4F16C0882311F096E911C0772321F0B9
:105C80009EE8872F762F05C0662371F096E8862F51
:105C900070E060E02AF09A95660F771F881FDAF7A8
:105CA000880F9695879597F9089512D180F09F37C0
:105CB00040F491110EF024C160E070E080E89FEBA9
:105CC000089526F41B16611D711D811D2BC045C052
:105CD000990F0008550FAA0BE0E8FEEF16161706FD
:105CE000E807F907C0F012161306E407F50798F065
:105CF000621B730B840B950B39F40A2661F0232B7E
:105D0000242B252B21F408950A2609F4A140A695F9
:105D10008FEF811D811D089597F99F6780E870E0DE
:105D200060E00895882371F4772321F09850872B41
:105D3000762F07C0662311F499270DC09051862B4A
:105D400070E060E02AF09A95660F771F881FDAF7F7
:105D5000880F9695879597F908959F3F49F0915040
:105D600028F4869577956795B7959F5F80389F4F04
:105D7000880F9695879597F908959FEF80EC089581
:105D8000DF93CF931F930F93FF92EF92DF927B01EC
:105D90008C01689405C0DA2EEF0196D1FE01E894DB
:105DA000A5912591359145915591AEF3EF01D8DD3F
:105DB000FE019701A801DA9479F7DF90EF90FF9048
:105DC0000F911F91CF91DF91089500240A94161628
:105DD000170618060906089500240A9412161306D9
:105DE000140605060895C9CF59D0E8F3E894EFEFFB
:105DF000BB273FE048EC5FE76B3D730784079507DF
:105E000008F1FF279F57B25A6A4D7F40894CF040F6
:105E100032F4BE556542704F8643FF4F0894EE1F23
:105E2000915030F0BB0F661F771F881FFF1FEBCF0D
:105E30009EE7882332F0BB0F661F771F881F9A9555
:105E4000C1F79395E09589CF092E0394000C11F4C6
:105E5000882352F0BB0F40F4BF2B11F460FF04C045
:105E60006F5F7F4F8F4F9F4F0895EF93E0FF06C006
:105E7000A2EA2AED3FE049EC5FEB72DDE5DF0F902F
:105E8000039401FC9058E3ECF0E0FAC157FD905800
:105E9000440F551F59F05F3F71F04795880F97FBEE
:105EA000991F61F09F3F79F08795089512161306A8
:105EB0001406551FF2CF4695F1DF08C016161706D7
:105EC0001806991FF1CF869571056105089408950C
:105ED000E5DFA0F0BEE7B91788F4BB279F3860F470
:105EE0001616B11D672F782F8827985FF7CF8695F4
:105EF00077956795B11D93959639C8F30895E89401
:105F0000BB2766277727CB0197F90895E1DE08F4D0
:105F10008FEF08955ADF19F05FDF09F02ECFFCCE26
:105F2000B901CA011ACF9F775F77B0DF98F3992341
:105F3000B9F35523B9F3FF27951758F4E52FE91B5B
:105F4000ED3070F75E3B10F0F1E41CC09034E0F4EB
:105F50000AC0E92FE51BED3028F79E3B10F0F1E475
:105F600011C0503488F4F9EA88232AF09A95660F14
:105F7000771F881FDAF744232AF05A95220F331F20
:105F8000441FDAF79F1B5F1BFF931F930F93FF9232
:105F9000EF9279018A01BB27AB2F9B01AC0196D010
:105FA0009701A801BF937B018C01AA27BA2FB901E1
:105FB000CA018CD0AF919701A801EF90FF900F918B
:105FC0001F91CEDC41DF01D14F9140FF089555274D
:105FD00047FD509509C09B01AC0160E070E080E88E
:105FE0009FE38DCD99CEB9CE59DFE8F39923D9F34C
:105FF000940F511DBBF39150504094F059F08823F9
:1060000032F0660F771F881F91505040C1F79E3FB6
:10601000510544F7880F911D9695879597F9089536
:106020005F3FACF0983E9CF0BB27869577956795CF
:10603000B79508F4B1609395C1F7BB0F58F711F409
:1060400060FFE8CF6F5F7F4F8F4F9F4FE3CF58CFF9
:1060500025DF58F19E5758F19851A0F0E9F098309B
:1060600020F5092E9927660F771F881F991F0A941C
:10607000D1F712C0062E672F782F8827985F11F46A
:10608000000C07C0993FB4F3869577956795939573
:10609000D9F7611D711D811D3EF490958095709515
:1060A00061957F4F8F4F9F4F0895689429CF27CFD9
:1060B0000BD0CACE8ADE28F08FDE18F0952309F0C7
:1060C0002BCE5BCE11241CCFE1DEA0F3959FD1F344
:1060D000950F50E0551F629FF001729FBB27F00D96
:1060E000B11D639FAA27F00DB11DAA1F649F6627EB
:1060F000B00DA11D661F829F2227B00DA11D621F3A
:10610000739FB00DA11D621F839FA00D611D221FF3
:10611000749F3327A00D611D231F849F600D211DD7
:10612000822F762F6A2F11249F5750408AF0E1F07A
:1061300088234AF0EE0FFF1FBB1F661F771F881FC3
:1061400091505040A9F79E3F510570F0E5CDD8CE53
:106150005F3FECF3983EDCF3869577956795B795AE
:10616000F795E7959F5FC1F7FE2B880F911D9695D8
:10617000879597F9089592DEE0F09E37D8F096392A
:10618000B8F49E3848F4672F782F8827985FF9CFA6
:1061900086957795679593959539D0F3B62FB1701D
:1061A0006B0F711D811D20F48795779567959395E9
:1061B000B9CDD3CDA5CE9F9317DE0F9007FCEE5F30
:1061C00054CE11F40EF4D9CDC8CD68DED0F39923A6
:1061D000D9F3CEF39F57550B87FF4BD05695979524
:1061E000B0E020F4660F771F881FBB1F1F930F932B
:1061F00000249001A0018001F001A0E80E0F1F1FF4
:106200000A1E511D601B710B8009B50B48F4600F0D
:10621000711F801DB51F0E1B1F0B0A0A510907C0F5
:106220002E0F3F1F4A1F0E0F1F1F0A1E511D660F04
:10623000771F881FBB1FA695F795E795F8F60617F9
:10624000170708065B07211D311D411D0F911F9186
:10625000B901842F9158880F9695879508959B01D1
:10626000AC0126CF35DE20F09F3708F449CE5ACD59
:1062700074CD91505040660F771F881FD2F7089554
:106280009F938F937F936F93FF93EF939B01AC0149
:106290000FDFEF91FF9174DD2F913F914F915F914F
:1062A00007CFA1E21A2EAA1BBB1BFD010DC0AA1F1E
:1062B000BB1FEE1FFF1FA217B307E407F50720F06F
:1062C000A21BB30BE40BF50B661F771F881F991FEA
:1062D0001A9469F760957095809590959B01AC0133
:0A62E000BD01CF010895F894FFCF2F
:00000001FF
